:0A13F00000010202030304040505D6
:10096500E4F515F514F513F512C20CC209C20BC254
:100975000A121C07120EA17E007F908E668F677586
:100985006E00756FA27564007565AC756C00756D4C
:10099500D37571007572FA90E680E030E70E8564D4
:1009A50068856569856C6A856D6B800C856C688565
:1009B5006D6985646A85656BEE54E07003020AD93A
:1009C5007516007517807E007F908E188F19C37479
:1009D500209FFF74019ECF2402CF3400FEE48F11C7
:1009E5008E10F50FF50EF50DF50CF50BF50AAF119B
:1009F500AE10AD0FAC0EAB0DAA0CA90BA80AC31215
:100A05000CBE502AE517250DF582E516350CF58344
:100A150074CDF0E4FAF9F8E50D2401F50DEA350C8D
:100A2500F50CE9350BF50BE8350AF50A80C0E4F558
:100A35000DF50CF50BF50AAF11AE10AD0FAC0EAB05
:100A45000DAA0CA90BA80AC3120CBE5035AE0CAFEB
:100A55000DE5192FF582E5183EF583E0FDE5172F25
:100A6500F582E5163EF583EDF0E4FAF9F8EF240199
:100A7500F50DEA3EF50CE9350BF50BE8350AF50AF7
:100A850080B585166685176774902480FF740034D9
:100A9500FFFEC3E56F9FF56FE56E9EF56EC3E569D5
:100AA5009FF569E5689EF568C3E56B9FF56BE56A9B
:100AB5009EF56AC3E5659FF565E5649EF564C3E546
:100AC5006D9FF56DE56C9EF56CC3E5729FF572E55E
:100AD500719EF571D2E843D82090E668E04409F0AC
:100AE50090E65CE0443DF0D2AF90E680E020E10581
:100AF500D20E121A8B90E680E054F7F0538EF8C2AE
:100B05000C300A05120470C20A300C291213FE506B
:100B150024C20C121B6D20091690E682E030E70412
:100B2500E020E1EF90E682E030E604E020E0E41228
:0A0B35001B15121CDC12101580C7FE
:010B3F002293
:1004700090E6B9E0700302054C1470030205F52400
:10048000FE700302068A24FB700302054614700303
:1004900002054014700302053414700302053A2467
:1004A0000560030206F6121CDE400302070290E616
:1004B000BBE024FE602C14604724FD6016146031FC
:1004C00024067066E56690E6B3F0E56790E6B4F062
:1004D000020702E56E90E6B3F0E56F90E6B4F00235
:1004E0000702E56890E6B3F0E56990E6B4F002072C
:1004F00002E56A90E6B3F0E56B90E6B4F00207021D
:1005000090E6BAE0FF121B41AA06A9077B01EA495F
:100510004B600DEE90E6B3F0EF90E6B4F002070208
:1005200090E6A0E04401F002070290E6A0E044015A
:10053000F0020702121CA4020702121CC8020702E2
:1005400012194A020702121C92020702121CE04012
:100550000302070290E6B8E0247F602B14603C247D
:100560000260030205EBA209E433FF25E0FFA20BC2
:10057000E4334F90E740F0E4A3F090E68AF090E691
:100580008B7402F0020702E490E740F0A3F090E6DB
:100590008AF090E68B7402F002070290E6BCE05409
:1005A0007EFF7E00E0D3948040067C007D018004C5
:1005B0007C007D00EC4EFEED4F24F0F58274133E7E
:1005C000F583E493FF3395E0FEEF24A1FFEE34E6DC
:1005D0008F82F583E0540190E740F0E4A3F090E6C9
:1005E0008AF090E68B7402F002070290E6A0E044E5
:1005F00001F0020702121CE2400302070290E6B873
:10060000E024FE601D2402600302070290E6BAE0C7
:10061000B40105C20902070290E6A0E04401F0021D
:10062000070290E6BAE0705990E6BCE0547EFF7E87
:1006300000E0D3948040067C007D0180047C007D36
:1006400000EC4EFEED4F24F0F58274133EF583E48A
:1006500093FF3395E0FEEF24A1FFEE34E68F82F5A1
:1006600083E054FEF090E6BCE05480FF1313135473
:100670001FFFE0540F2F90E683F0E04420F00207C4
:100680000290E6A0E04401F08078121CE4507390E0
:10069000E6B8E024FE60202402706790E6BAE0B479
:1006A0000104D209805C90E6BAE06402605490E6EE
:1006B000A0E04401F0804B90E6BCE0547EFF7E0059
:1006C000E0D3948040067C007D0180047C007D00A6
:1006D000EC4EFEED4F24F0F58274133EF583E49367
:1006E000FF3395E0FEEF24A1FFEE34E68F82F58321
:1006F000E04401F0800C120122500790E6A0E04493
:0907000001F090E6A0E04480F055
:0107090022CD
:030033000213FABB
:0413FA0053D8EF32A3
:101C0700758CE0758AC0E58954F04401F589758EB5
:081C170003D28CD2A9D2AF2246
:03000B00020CF5EF
:100CF500C0E0C0F0C083C082C0D075D000C000C0C5
:100D050001C002C003C004C005C006C007758CE061
:100D1500758AC0D28CE47F607EEAFDFCAB60AA5F79
:100D2500A95EA85DC3120CBE501DAF60AE5FAD5E7F
:100D3500AC5DE4FAF9F8EF2401F560EA3EF55FE908
:100D45003DF55EE83CF55DE47F01FEFDFCAB60AA88
:100D55005FA95EA85DC3120CBE70097570827563CC
:100D650001853E62E47F02FEFDFCAB60AA5FA95EE1
:100D7500A85DC3120CBE700D90E678E04480F0903B
:100D8500E679E570F0E47F03FEFDFCAB60AA5FA9A0
:100D95005EA85DC3120CBE700690E679E563F0E4CB
:100DA5007F04FEFDFCAB60AA5FA95EA85DC3120CC3
:100DB500BE700690E679E562F0E47F05FEFDFCABCA
:100DC50060AA5FA95EA85DC3120CBE700790E678A5
:100DD500E04440F0E52C2401FFE4352BFEE4FCFD66
:100DE500AB60AA5FA95EA85DC3120CBE70097570E1
:100DF500827563017562F0E52C2402FFE4352BFE54
:100E0500E4FCFDAB60AA5FA95EA85DC3120CBE70D1
:100E15000D90E678E04480F090E679E570F0E52CF9
:100E25002403FFE4352BFEE4FCFDAB60AA5FA95E5D
:100E3500A85DC3120CBE700690E679E563F0E52C5B
:100E45002404FFE4352BFEE4FCFDAB60AA5FA95E3C
:100E5500A85DC3120CBE700690E679E562F0E52C3C
:100E65002405FFE4352BFEE4FCFDAB60AA5FA95E1B
:100E7500A85DC3120CBE700990E678E04440F0C24C
:100E85008CD007D006D005D004D003D002D001D035
:0C0E950000D0D0D082D083D0F0D0E0326A
:100090001201000200000040181685A200000102B3
:1000A00000010A06000200000040010009022700CA
:1000B000010100A0FA0904000003FF000000070589
:1000C0000102400000070586020002000705020247
:1000D00000020009022700010100A0FA0904000043
:1000E00002FF00000007050102400000070586022C
:1000F00040000007050202400000040309040E034B
:10010000530048002D0049004D00470014034900EA
:100110004D00470032005300200020002000200046
:020120000000DD
:03004300021400A4
:0300530002140094
:10140000021C1F00021C7C00021C6600021C37002C
:10141000021981000219B80002008F00021CE600C8
:10142000021CE700021CE800021CE90002070A0097
:10143000021CEA00021CEB00021CEC00021CED0086
:10144000021CEE00021CE600021CEF00021CF00071
:10145000021CF100021CF200021CF300021CF4004A
:10146000021CF500021CE600021CE600021CE6005D
:10147000021CF600021CF700021CF800021CF90016
:10148000021CFA00021CFB00021CFC00021CFD00F6
:10149000021CFE00021CFF00021D0000021D0100D4
:1014A000021D0200021D0300021D0400021D0500B2
:0814B000021D0600021D0700E9
:101B150090E682E030E004E020E60B90E682E030DB
:101B2500E119E030E71590E680E04401F07F147E8E
:0C1B35000012190490E680E054FEF0223B
:101B6D0090E682E044C0F090E681F04387010000EA
:041B7D000000002242
:101A8B00300E0990E680E0440AF0800790E680E093
:101A9B004408F07FDC7E0512190490E65D74FFF0BC
:0F1AAB0090E65FF05391EF90E680E054F7F02261
:021B4100A907F2
:101B4300AE71AF728F828E83A3E064037017AD0111
:101B530019ED7001228F828E83E07C002FFDEC3E15
:091B6300FEAF0580DF7E007F006B
:011B6C002256
:101904008E1C8F1D90E600E054187012E51D240112
:10191400FFE4351CC313F51CEF13F51D801590E689
:1019240000E05418FFBF100BE51D25E0F51DE51C74
:1019340033F51CE51D151DAE1C7002151C4E60050B
:06194400121B8180EE225F
:101B81007400F58690FDA57C05A3E582458370F977
:011B91002231
:1018B300C106C10802371A000229000002550000C0
:1018C300025703F7024E0000022600000235000013
:1018D30001390101340101450001530001400001B8
:1018E30054000151000161A0045900000000C10728
:1018F300C104C1030122CF013F00C100C101C105E1
:101BD500200E0B53227FAD227F801216A1224322B5
:091BE50080AD227F801216A122BE
:101BEE00300E0B5322FEAD227F801216A12243220D
:091BFE0001AD227F801216A12224
:101BB600300E0E7D017F031216A190E60174CBF064
:0F1BC60022E4FD7F031216A190E6017443F02282
:100EA10090E6007412F090E6017443F000000090A7
:100EB100E61074A0F000000000000090E612F000BF
:100EC1000000E490E613F000000090E61474E0F0F6
:100ED100000000E490E615F000000090E604748044
:100EE100F00000007402F00000007406F000000041
:100EF100E4F000000090E60274E6F000000090E6E5
:100F01000374F8F000000090E670E04440F0000047
:100F110000E490E609F000000043B20F90E61804E7
:100F2100F00000007411F000000090E61A7409F05E
:100F3100000000E490E671F090E672F075B203757E
:100F4100B6FF75B4BFC2A5C28CC20E121BD57F6499
:100F51007E00121C4FD20E121BD5D281C20290E626
:100F61005EE04408F0000000E490E68DF0D2A312A8
:100F71001CD87522CFC20E121BEE7D507F011216B6
:100F8100A17D227F021216A17D017F041216A17D8F
:100F9100017F081216A1E4FD7F101216A17D647F66
:100FA100201216A17D1A7F401216A17DFF7F8012AB
:100FB10016A17D807C00E4FF12156F7DFF7C007F10
:100FC1000112156F7D0F7C007F0312156F7D1F7C51
:100FD100007F0412156F7D1F7C007F0512156F7D48
:100FE1001F7C007F0612156F7D1F7C007F07121585
:100FF1006FC200C201C2A4D2A7121CD07BF07D0334
:101001007F82121ABA7BF07D017F82121ABAD20E48
:04101100121BB622D6
:101015002006030210D830000BAD24AC237F01124B
:10102500156FC20030012AE53AFD7C007F041215D8
:101035006FE53BFD7C007F0512156FE53CFD7C00EF
:101045007F0612156FE53DFD7C007F0712156FC207
:1010550001300518533F075322C7E53F75F008A433
:101065002522F522FD7F801216A1C20530042CAD84
:10107500497F041216A1AD507F021216A1AD417F22
:10108500F01216A1AD427FF11216A1AD437FF21207
:1010950016A1AD447FF31216A1C204E554146012E3
:1010A50014601A2402702130A6032007FA1214B81E
:1010B500806F30A6032007FA121236806430A6032B
:1010C5002007FA121316805930A6032007FA1214C6
:1010D500B8804EE4FAF9F8E55C2401F55CEA355B85
:1010E500F55BE9355AF55AE83559F559E47F64FE5B
:1010F500FDFCAB5CAA5BA95AA859C3120CBE7003D0
:10110500121861E47F207E4EFDFCAB5CAA5BA95AF8
:10111500A859D3120CBE4009E4F55CF55BF55AF508
:0911250059E551B40102C2062291
:0213FE00D322F8
:021CDC00D32211
:021CDE00D3220F
:10194A0090E680E030E71590E6247402F00000008B
:10195A00E490E625F0000000D2028013E490E62429
:10196A00F000000090E6257440F0000000C20290EA
:07197A00E6BAE0F552D322AA
:101C920090E740E552F0E490E68AF090E68B04F09B
:021CA200D3224B
:081CC80090E6BAE0F528D322F2
:101CA40090E740E528F0E490E68AF090E68B04F0B3
:021CB400D32239
:021CE000D3220D
:021CE200D3220B
:021CE400D32209
:1001220090E6B9E0120CCF0148B302C7B503A8B6F6
:100132000194BA01B2BB01EBBC0212BD03E0C204DE
:1001420026C90000046EE490E68AF090E68BF00087
:10015200000090E6047480F0000000C20E121BD56D
:1001620090E6047406F0000000E4F0FF7E0112192C
:1001720004D20E121BD57F0A7E001219047D807CE8
:1001820000E4FF12156FD206752501C203D20602E2
:10019200046EE490E68AF090E68BF090E6A0E02010
:1001A200E1F990E68BE0F51A000000C20602046E47
:1001B200E490E68AF090E68BF090E6A0E020E1F988
:1001C20090E68BE0F51A00000090E740E0F546A3C8
:1001D200E0FEA3E07C002400F548EC3EF547AD4884
:1001E200FCAF4612156F02046EE490E68AF090E6C8
:1001F2008BF090E6A0E020E1F990E68BE0F51A00A2
:10020200000090E740E0FFA3E0FD1216A102046E99
:10021200E490E68AF090E68BF090E6A0E020E1F927
:1002220090E68BE0F51A00000090E740E0F52DA380
:10023200E0F52FA3E0F52EE52FFE7C00E4252EFF4E
:10024200EC3EFEE48F4D8E4CF54BF54A7F0AFEFDE7
:10025200AB4DAA4CA94BA84AC3120CBE500575530C
:1002620001801BE54D24F6F54DE54C34FFF54CE5D8
:100272004B34FFF54BE54A34FFF54AE4F553E4FF0E
:10028200FEE54BFDE4FCFB7A01F9F8120C2CE4FBD1
:100292007A01F9F8120C2C8F2DE4FFE54CFEE4FDF7
:1002A200FCFB7A01F9F8120C2C8F2FE54DFFE48F3D
:1002B2002E90E743E0FEA3E07C002400F536EC3EFE
:1002C200F53502046EE490E68AF090E68BF090E653
:1002D200A0E020E1F990E68BE0F51AE4F51B74400A
:1002E200251BF582E434E7F583E0FF7400251BF556
:1002F20082E43427F583EFF0051BE51BB440DF9061
:100302002707E0FD7F401216A1902708E0FD7F201D
:100312001216A1902711E0FD7F101216A19027124C
:10032200E0FD7F081216A1902720E0F54590272EC8
:10033200E0F54090273AE0F56190273CE0F554A3C0
:10034200E0F551902721E0FF70035322BFEFB40183
:10035200035322BFEFB402035322BFEFB40303439C
:10036200224090272AE070055322FD800343220297
:10037200AD227F801216A1AD617F011216A17D0F01
:100382007C007F0312156F7D807C00E4FF12156FE5
:1003920090273BE07008C20E121BB602046ED20E0A
:1003A200121BB602046EE4F51B7400251BF582E4F1
:1003B2003427F583E0FF7440251BF582E434E7F52A
:1003C20083EFF0051BE51BB440DF000000E490E67C
:1003D2008AF000000090E68B7440F002046E90E711
:1003E2004074ABF0A37408F0A37403F0A3741BF081
:1003F200A37402F0A37454F0A37401F0A304F0A355
:1004020074B8F0300205E4A3F0800690E74974FF67
:10041200F0000000E490E68AF000000090E68B74A1
:100422000AF08048E490E68AF090E68BF090E6A02D
:10043200E020E1F990E68BE0F51A90E740E054F015
:10044200FFC4540F24F0FB7D017F82121ABA90E799
:1004520041E075F00AA4FFAEF012190490E740E003
:0D04620024F0540FFB7D017F82121ABAC3F3
:01046F00226A
:101C1F00C0E0C083C082D20A5391EF90E65D740199
:081C2F00F0D082D083D0E03236
:101C6600C0E0C083C0825391EF90E65D7404F0D06B
:061C760082D083D0E032B1
:101C7C00C0E0C083C0825391EF90E65D7402F0D057
:061C8C0082D083D0E0329B
:10198100C0E0C083C08290E680E030E70E856468E5
:10199100856569856C6A856D6B800C856C68856D64
:1019A1006985646A85656B5391EF90E65D7410F00B
:0719B100D082D083D0E032A8
:101C3700C0E0C083C082D20C5391EF90E65D740878
:081C4700F0D082D083D0E0321E
:1019B800C0E0C083C08290E680E030E70E856468AE
:1019C800856569856C6A856D6B800C856C68856D2D
:1019D8006985646A85656B5391EF90E65D7420F0C4
:0719E800D082D083D0E03271
:01008F00323E
:011CE60032CB
:011CE70032CA
:011CE80032C9
:011CE90032C8
:10070A00C0E0C0F0C083C082C0D075D000C000C0B5
:0D071A0001C002C003C004C005C006C00736
:10072700C2AF90E6A1E020E1F990E780E0FF120C6C
:10073700CF07600007800207960307AD04080B0583
:10074700081F06082A07084908090C09077BFD073F
:1007570070FE0766FF000009367525000209367529
:100767002500D203C20602093690E781E024FF92F2
:1007770007020936C28C02093690E781E0FEA3E042
:100787007C002400F524EC3EF523D20002093690C4
:10079700E781E0F53AA3E0F53BA3E0F53CA3E0F5FC
:1007A7003DD20102093690E781E0F52DA3E0F52F50
:1007B700A3E0F52EAF2FE4FCFDFEFB7A01F9F8125A
:1007C7000BA1C004C005C006C007AF2DE4FCFDFEA9
:1007D700FBFA7901F8120BA1D003D002D001D000A7
:1007E700EF2BFBEE3AFAED39F9EC38F8E4FCFDFEB5
:1007F700EB252EF533EE3AF532ED39F531EC38F5D8
:100807003002093690E781E0FEA3E07C002400F582
:1008170036EC3EF53502093690E781E0F53FD20523
:1008270002093690E781E0F549A3E0F550A3E0F52A
:1008370041A3E0F542A3E0F543A3E0F544D2040267
:100847000936E4FF74802FF582E434E7F583E0FE90
:1008570074002FF582E43427F583EEF00FBF40E4F0
:10086700902707E0FD7F401216A1902708E0FD7F43
:10087700201216A1902711E0FD7F101216A19027D4
:1008870012E0FD7F081216A1902720E0F54590277A
:100897002EE0F54090273AE0F56190273CE0F554CB
:1008A700A3E0F551902721E0FF70035322BFEFB477
:1008B70001035322BFEFB402035322BFEFB4030374
:1008C70043224090272AE070055322FD80034322EC
:1008D70002AD227F801216A1AD617F011216A17DA4
:1008E7000F7C007F0312156F7D807C00E4FF1215DB
:1008F7006F902745E07007C20E121BB68031D20EEB
:10090700121BB6802AD28C90E781E0540FF53EA3E4
:10091700E0FEA3E07C002400FFEC3EC313F52BEFC1
:1009270013F52C756000755F00755E00755D00003E
:10093700000090E68DE4F05391EF90E65FE0440805
:03094700F0D2AF3C
:10094A00D007D006D005D004D003D002D001D00001
:0B095A00D0D0D082D083D0F0D0E032AB
:011CEA0032C7
:011CEB0032C6
:011CEC0032C5
:011CED0032C4
:011CEE0032C3
:011CEF0032C2
:011CF00032C1
:011CF10032C0
:011CF20032BF
:011CF30032BE
:011CF40032BD
:011CF50032BC
:011CF60032BB
:011CF70032BA
:011CF80032B9
:011CF90032B8
:011CFA0032B7
:011CFB0032B6
:011CFC0032B5
:011CFD0032B4
:011CFE0032B3
:011CFF0032B2
:011D000032B0
:011D010032AF
:011D020032AE
:011D030032AD
:011D040032AC
:011D050032AB
:011D060032AA
:011D070032A9
:101C4F00AD07AC06ED25E0FDEC33FCED4C6007ED88
:071C5F001D70011C80F5223D
:10172600E545B40105D20E121BEE752501E52D75B2
:10173600F040A485F01AF51BAF257E00AC1AAD1B50
:10174600120B8FD3EF9400EE940040117FDE7E03E0
:10175600121904E51B151B7002151A80DB751A0099
:10176600852F1BAF257E00AC1AAD1B120B8FD3EF56
:101776009400EE940040117FFD7E00121904E51BD3
:10178600151B7002151A80DBAF2E7E00121904E5B8
:0917960045B40105C20E121BEE60
:01179F002227
:041CD80075B1EE22D2
:1018610075B16F00000000000075B16E000000004E
:10187100000075B1EE00000000000075B1EC000041
:101881000000000075B1FC00000000000075B17C93
:1018910000000000000075B17D000000000000752F
:1018A100B16D00000000000075B16F000000000084
:0218B100002213
:10180B0075B16F00000000000075B16E00000000A4
:10181B00000075B1EE00000000000075B1EC000097
:10182B0000000000C2A775B1FC00000000000075AD
:10183B00B17C00000000000075B17D0000000000CD
:10184B0000D2A775B16D00000000000075B16F00EC
:06185B0000000000002265
:101CB600E4FFFE1218610FBF00010EBE04F5BF1A45
:011CC600F22B
:011CC70022FA
:1017A00075B16F00000000000075B16E0000000010
:1017B000000075B1EE00000000000075B1EC000003
:1017C0000000000075B1FC00000000000075B17C55
:1017D00000000000000075B17D00000000000075F1
:1017E000B16D0000000000007F017E00121C4F75EB
:1017F000B10D00000000000075B10F0000000000F6
:0B1800000075B16F0000000000002226
:0F008000C2A77F037E00121C4FD2A7121C4F2273
:06156F008C1C8D1DA90774
:10157500530107C2A37F0A7E00121C4FC2A2121C90
:101585004FD2A1121C4FC2A1E4FBFAAF03E9A80791
:10159500088002C313D8FC30E004D2A28002C2A2A4
:1015A5007F0A7E00121C4FD2A1121C4FC2A1121C31
:1015B5004F0BBB00010AEB64034A70CFC2A27F0A3E
:1015C5007E00121C4FD2A1121C4FC2A1E4FAFBAF40
:1015D50003E51DAE1CA807088005CEC313CE13D89E
:1015E500F930E004D2A28002C2A27F0A7E00121C5A
:1015F5004FD2A1121C4FC2A1121C4F0BBB00010AF6
:0F160500EB640B4A70C9D2A37F0A7E00121C4F00
:0116140022B3
:0416A1008F1CA905EC
:1016A500C2A07F017E00121C4FE4FBFAAF03E9A83C
:1016B50007088002C313D8FC30E004D2A28002C21E
:1016C500A27F017E00121C4FD2A1121C4FC2A11293
:1016D5001C4F0BBB00010AEB64084A70CFE4FAFB10
:1016E500AF03E51CA807088002C313D8FC30E0044B
:1016F500D2A28002C2A27F017E00121C4FD2A1128B
:101705001C4FC2A1121C4F0BBB00010AEB64084A17
:1017150070CED2A07F017E00121C4FC2A0121C4FBA
:0117250022A1
:101ABA00AC07AA0590E678E04480F090E679ECF06D
:101ACA007F647E00121C4FEAF0121C4FEBF0121CCE
:0E1ADA004F90E678E04440F07F64121C4F22EB
:101B920090272AE07019432202AD227F801216A1FB
:101BA200D2A5C2A55322FDAD227F801216A122D258
:041BB200A5C2A52201
:1014B80085334D85324C85314B85304AE4FFFEE556
:1014C8004BFDE4FCFB7A01F9F8120C2CE4FB7A01E1
:1014D800F9F8120C2C8F2DE4FFE54CFEE4FDFCFB23
:1014E8007A01F9F8120C2C8F2FE54DFFE48F2EFFAF
:1014F800FEFDFCAB4DAA4CA94BA84AD3120CBE402A
:101508000375B1FF121B92121726E4FFFEFDFCAB18
:101518004DAA4CA94BA84AD3120CBE4003121CB6C4
:101528001217A0121861E4FBFAC3EB940AEA64806C
:1015380094805004D2808002C280C2817F017E00E4
:10154800121C4F2083033003FAD281EBB53609EA27
:10155800B5350512180B80031218610BBB00010A80
:06156800BA04C6BB1AC361
:01156E00225A
:1012360085334D85324C85314B85304AE47F06FE39
:10124600FDFCAB4DAA4CA94BA84AC3120CBE5005D7
:10125600755301801BE54D24FAF54DE54C34FFF539
:101266004CE54B34FFF54BE54A34FFF54AE4F553BC
:10127600E4FFFEE54BFDE4FCFB7A01F9F8120C2CC9
:10128600E4FB7A01F9F8120C2C8F2DE4FFE54CFEF5
:10129600E4FDFCFB7A01F9F8120C2C8F2FE54DFFCB
:1012A600E48F2EE553B40103121CB6121B921200F2
:1012B6008075B1FF121726E5537003121CB612177C
:1012C600A0121861D280E545B401057F32121AE8F2
:1012D600C280E545B401057FC8121AE8E4FBFAC3EB
:1012E600EB940AEA648094805004D2808002C28023
:1012F600C2817F017E00121C4F2083033003FAD285
:0F130600811218610BBB00010ABA04D3BB1AD0C5
:0113150022B5
:1013160085334D85324C85314B85304AE4FFFEE5F9
:101326004BFDE4FCFB7A01F9F8120C2CE4FB7A0184
:10133600F9F8120C2C8F2DE4FFE54CFEE4FDFCFBC6
:101346007A01F9F8120C2C8F2FE54DFFE48F2E123F
:101356001B92E4FFFEFDFCAB4DAA4CA94BA84AD359
:10136600120CBE400375B1FF121726E4FFFEFDFC0A
:10137600AB4DAA4CA94BA84AD3120CBE4003121C73
:10138600B61217A0121861E4FBFA1218610BBB0023
:10139600010ABA01F5BB1CF2E4FAFBC3EB940AEAB4
:1013A600648094805004D2808002C280C2817F0112
:1013B6007E00121C4F2083033003FAD281EBB53630
:1013C60009EAB5350512180B80031218610BBB002C
:1013D600010ABA01C6BBE0C3E4FAFB1218610BBBF3
:0913E60000010ABA01F5BB1EF278
:0113EF0022DB
:101AE8008F1A5322FBAD227F801216A1E51A6012CD
:101AF800C2817F017E00121C4F3083FDD281151AEE
:0D1B080080EA432204AD227F801216A12244
:081CD000E4F578D2E9D2AF225D
:1019EF0090E678E020E6F9C2E990E678E04480F0EE
:1019FF00EF25E090E679F090E678E030E0F990E6B8
:101A0F0078E04440F090E678E020E6F990E678E060
:061A1F0030E1D6D2E922FD
:101A5900A90790E678E020E6F9E578702390E67822
:101A6900E04480F0E925E090E679F08D73AF03A9B1
:101A7900077574018A758976E4F577757801D3223B
:021A8900C32276
:101A2500A90790E678E020E6F9E578702590E67854
:101A3500E04480F0E925E0440190E679F08D73AF4C
:101A450003A9077574018A758976E4F577757803B6
:041A5500D322C322B3
:03004B0002112E71
:10112E00C0E0C083C082C085C084C086758600C002
:10113E00D075D000C000C001C002C003C006C007F9
:10114E0090E678E030E20675780602121890E6789E
:10115E00E020E10CE578640260067578070212184B
:10116E00E57824FE605F14603624FE7003021209D7
:10117E0024FC700302121524086003021218AB74CB
:10118E00AA75A976AF7705778F82758300120B400B
:10119E0090E679F0E57765737070757805806B90E1
:1011AE00E679E0AB74AA75A976AE778E8275830068
:1011BE00120B6D757802E5736401704E90E678E05F
:1011CE004420F08045E57324FEB5770790E678E07D
:1011DE004420F0E57314B5770A90E678E04440F0C9
:1011EE0075780090E679E0AB74AA75A976AE778E25
:1011FE0082758300120B6D0577800F90E678E044C0
:10120E0040F075780080037578005391DFD007D0D9
:10121E0006D003D002D001D000D0D0D086D084D05A
:08122E0085D082D083D0E032AC
:03000000021615D0
:0C161500787FE4F6D8FD75817802165C41
:100B4000BB010CE58229F582E5833AF583E022506A
:100B500006E92582F8E622BBFE06E92582F8E222B4
:0D0B6000E58229F582E5833AF583E49322CE
:100B6D00F8BB010DE58229F582E5833AF583E8F0BE
:100B7D00225006E92582C8F622BBFE05E92582C86A
:020B8D00F22252
:100B8F00EF8DF0A4A8F0CF8CF0A428CE8DF0A42E7A
:020B9F00FE2234
:100BA100E88FF0A4CC8BF0A42CFCE98EF0A42CFCF3
:100BB1008AF0EDA42CFCEA8EF0A4CDA8F08BF0A471
:100BC1002DCC3825F0FDE98FF0A42CCD35F0FCEBD0
:100BD1008EF0A4FEA9F0EB8FF0A4CFC5F02ECD3995
:0F0BE100FEE43CFCEAA42DCE35F0FDE43CFC2202
:100BF00075F008758200EF2FFFEE33FECD33CDCCBC
:100C000033CCC58233C5829BED9AEC99E58298403E
:100C10000CF582EE9BFEED9AFDEC99FC0FD5F0D61B
:100C2000E4CEFBE4CDFAE4CCF9A88222B800C1B945
:100C30000059BA002DEC8BF084CFCECDFCE5F0CB83
:100C4000F97818EF2FFFEE33FEED33FDEC33FCEBBC
:100C500033FB10D703994004EB99FB0FD8E5E4F977
:100C6000FA227818EF2FFFEE33FEED33FDEC33FC64
:100C7000C933C910D7059BE99A4007EC9BFCE99A58
:100C8000F90FD8E0E4C9FAE4CCFB2275F010EF2F9D
:100C9000FFEE33FEED33FDCC33CCC833C810D7079D
:100CA0009BEC9AE899400AED9BFDEC9AFCE899F8D8
:0E0CB0000FD5F0DAE4CDFBE4CCFAE4C8F9226B
:100CBE00EB9FF5F0EA9E42F0E99D42F0E89C45F08C
:010CCE002203
:100CCF00D083D082F8E4937012740193700DA3A3B4
:100CDF0093F8740193F5828883E4737402936860C8
:060CEF00EFA3A3A380DFC8
:10162100020965E493A3F8E493A34003F68001F271
:1016310008DFF48029E493A3F85407240CC8C333CA
:10164100C4540F4420C8834004F456800146F6DF99
:10165100E4800B01020408102040809018B3E47E5E
:10166100019360BCA3FF543F30E509541FFEE4938E
:10167100A360010ECF54C025E060A840B8E493A355
:10168100FAE493A3F8E493A3C8C582C8CAC583CA80
:10169100F0A3C8C582C8CAC583CADFE9DEE780BE38
:0119030000E3
:00000001FF
